:10000000E12808303B190130A300A2013E0884001A
:100010003C0843203C08800484130005FF3E3B1D40
:10002000A20C3B19A20D32306920A30B082822082C
:100030000314DC28A20008303B190130A300A20CF5
:100040003E0884003C0843203C08031880043C30F0
:1000500069203C088004A30B1F280314DC28BB1C68
:10006000DC283528BB003B1CDC283E0884003C080B
:1000700043200130A100F4306A203C0880040130A4
:10008000A100F4306A28FF3A8005462884178005CD
:10009000DC288000DC2883169B001C141A08DC284E
:1000A00083169A001C1555309D00AA309D009C14A3
:1000B0009C1858281C11DC28A301A200FF30A207BD
:1000C000031CA307031CDC280330A100DF306A20D7
:1000D0005E28A101E83EA000A109FC30031C7328A2
:1000E000A00703187028A0076400A10F702820182B
:1000F0007928A01C7D2800007D280800013EA7006B
:100100000A30A200A301C020A70B832824080800FE
:100110000310A10CA00CFF3E031888282008DC283F
:10012000A101A301A2000230A528A2000330A52846
:10013000A101A301A2000130A528A2000630A52834
:10014000A2000430A528A2000530A800230821023F
:10015000031DAC28220820020430031801300319C3
:1001600002302805031DFF30DC280038031DFF3056
:100170000405031DFF30DC280404031DFF30DC28C8
:10018000A501A4011030A600210DA40DA50D220883
:10019000A4022308031C230FA5020318D628220853
:1001A000A40723080318230FA5070310A00DA10D12
:1001B000A60BC4282008DC288313031383126400D1
:1001C0000800CC01CD01C601C701CB010130D1002F
:1001D0001630D2005011D010831686118312861566
:1001E00083130313831207309F00031383168117B1
:1001F0008112831283163F30920083123F309500A4
:10020000043092008316860183120F309700831604
:100210008601831286018316051383120513831644
:1002200005108510831205148514831686170A306D
:1002300083125C206400861B1F29D0153529831684
:100240008613831286130230A100BC306A20831605
:10025000861786173C30831269206400861B31297B
:10026000D0116400861F3529D0156400D0193B29B0
:1002700001304B20D20064005208FF3C031D42298C
:100280001930D20064000A305202031849290A309A
:10029000D20064005B305202031C50295A30D20055
:1002A00002304B20C70003304B20C6004608A00098
:1002B0004708A100FF30A300FF30A320031D6529DC
:1002C0002730A30010305D20C6254608A00047084F
:1002D000A1004030A200A301C020C2002108C30039
:1002E0006400D019EC290630BE008030BC0001301B
:1002F0003220CC301A2044301A202F208316861743
:100300008312C001C101C00A0319C10A19305C205F
:100310000630BE008030BC00043032200120C8000E
:100320002F204008A0004108A100A30128309A20F6
:10033000031DEC2964004808003C0319832906309A
:10034000BE008030BC0001303220CC301A20BE30DC
:100350001A202F200630BE008030BC000230322030
:100360000120C4000120C5000120C8000120C800F0
:100370000120C8000120C8000120C8000120CA00D7
:100380002F206400F9304502031CC929C401C501AE
:10039000D2294408A0004508A10004308B20C400E5
:1003A0002108C5004408A0004508A100A30155305C
:1003B000A320031DDE290130C400C5014408A000AC
:1003C0004508A10001307E20CC004408A00045086B
:1003D000A10000307E20CD006400D01D2A2A1730F5
:1003E000D200831605118511831205118515013080
:1003F000A3002C305D200A305C20831605166400B3
:100400008312051A052AC90A062AC90164000A309E
:100410004902031CFB290511851105158511C00131
:10042000C1010A305C20C00A0319C10A83160516EF
:1004300003108312470CB300460CB2004008A00022
:100440004108A1003308A30032089D20031D112A92
:10045000051185110030D0190130A0000030902026
:10046000B200FB305207B400FF300318013EB50064
:100470004408A0004508A1003508A3003408A020C6
:10048000B400320884003408B520B400B50064001C
:10049000340835040319672A831605118511831260
:1004A0000515851164305C200A305C208316051622
:1004B00064008312051A5E2AC90A5F2AC901640012
:1004C0000A304902031C542A0511851150150030C9
:1004D000D0190130A00000309020B2000530520742
:1004E000B400B501B50D4408A0004508A1003508C9
:1004F000A30034089A20B400320884003408B520E0
:10050000B400B5006400340835040319A22A831628
:100510000511851183120511851564305C200A30A0
:100520005C208316051664008312051A992AC90AED
:100530009A2AC90164000A304902031C8F2A051156
:100540008511D014831686010510851005136400EB
:1005500083124908803C031DB12ACA228510051464
:10056000062464004908003C031DB92A05108514BF
:10057000182464005018C82A64004908A03C031DD0
:10058000C22A051064004908203C031DC82A8510B2
:10059000C90AA22A64001E304E020318D12ACE0ACC
:1005A0000800640029304F02031CD72AD124831687
:1005B0000614861406150517831205108510CE0142
:1005C000003006180130A00001309020B200003049
:1005D00086180130A00001309020B4003208840059
:1005E0003408B520B400B5000030051B0130A00070
:1005F00001309020B6003408350484003608B52058
:10060000B600B700003006190130A000013090207C
:10061000B8003608370484003808B520B800B9009F
:100620006400380839040319172BCF0A0800CF01DA
:10063000640006183F2BD1036400013051020318F7
:10064000232B0130D100FF305107B200FF300318D7
:10065000013EB3003208A0003308A10001307E2023
:10066000CC00FF305107B200FF300318013EB30049
:100670003208A0003308A10000307E20CD006400C5
:100680008618662BD10A64000C305102031C4A2BD9
:100690000B30D100FF305107B200FF300318013E8C
:1006A000B3003208A0003308A10001307E20CC0046
:1006B000FF305107B200FF300318013EB30032088B
:1006C000A0003308A10000307E20CD006400061990
:1006D000882B0530D20264000A3052020318722BB4
:1006E0000A30D200831601309B008312520850203A
:1006F0005208A000A10101307E20CC005208A000C9
:10070000A10100307E20CD006400D01D882B512433
:100710006400051BAA2B0530D2076400603052022A
:10072000031C942B5F30D200831601309B00831290
:10073000520850205208A000A10101307E20CC00B8
:100740005208A000A10100307E20CD006400D01D21
:10075000AA2B912464005108013C031DB22B3F30A9
:100760009500042C64005108023C031DBA2B243070
:100770009500042C64005108033C031DC22B223059
:100780009500042C64005108043C031DCA2B203042
:100790009500042C64005108053C031DD22B1C302D
:1007A0009500042C64005108063C031DDA2B183018
:1007B0009500042C64005108073C031DE22B143003
:1007C0009500042C64005108083C031DEA2B1030EE
:1007D0009500042C64005108093C031DF22B0C30D9
:1007E0009500042C640051080A3C031DFA2B0830C4
:1007F0009500042C640051080B3C031D022C0430AE
:100800009500042C3F309500501408004C08093C1A
:10081000031C182C04308A004C0882072A2C2E2C2A
:10082000322C362C3A2C3E2C422C462C4A2C4D2C69
:100830004D08093C031C2A2C04308A004D0882070D
:100840002A2C2E2C322C362C3A2C3E2C422C462C88
:100850004A2C4D2C4030860005130800713086006C
:100860000517080024308600051308003030860084
:1008700005130800113086000517080012308600A5
:10088000051308000230860005130800703086004A
:1008900005170800860105130800103086000513AF
:1008A00008006400D01C552C080050118316051157
:1008B000851183120510851005118515C001C10130
:1008C000C9010A305C20C00A0319C10A8316051643
:1008D00064008312051A6E2CC90A6F2CC9014008E6
:1008E000A0004108A1004308A30042089A20B200DA
:1008F0004908A00003309820B4003208840034086E
:10090000BC20B400B5006400340835040319612C20
:10091000640004304902031C8E2CD014051185118B
:1009200008006400501D952C0800D0108316051196
:10093000851183120510851005158511C001C101AF
:10094000C9010A305C20C00A0319C10A83160516C2
:1009500064008312051AAE2CC90AAF2CC9014008E5
:10096000A0004108A1004308A30042089A20B20059
:100970004908A00003309820B400320884003408ED
:10098000BC20B400B5006400340835040319A12C60
:10099000640004304902031CCE2C5015051185114A
:1009A0000800051085106400D01DD92CCF0150100F
:1009B00008000630BE008030BC0001303220CC3050
:1009C0001A2044301A202F20831686178312C00164
:1009D000C101C00A0319C10A851005140624093093
:1009E000A100C4306A2005101B30A10058306A20D5
:1009F0000510851418240930A100C4306A20851020
:100A00001930A10064306A200630BE008030BC007E
:100A1000043032200120C8002F204008A0004108E7
:100A2000A100A30132309D20031D172D0800640092
:100A30004808003C0319E92C0630BE008030BC0099
:100A400001303220CC301A20BE301A202F20063040
:100A5000BE008030BC00023032200120C4000120E2
:100A6000C5000120C8000120C8000120C8000120E5
:100A7000C8000120C8000120CA002F206400F930FE
:100A80004502031C462DC401C5014F2D4408A0009A
:100A90004508A10004308B20C4002108C5000230A5
:100AA0005207B200B301B30D4408A0004508A100ED
:100AB0003308A30032089D20031D5F2D5124FE3012
:100AC0005207B200FF300318013EB3004408A000F3
:100AD0004508A1003308A30032089520031D712D9D
:100AE000912404305207B200B301B30D4408A000B2
:100AF0004508A1003308A30032089D20031D812D65
:100B00005124FC305207B200FF300318013EB300FD
:100B10004408A0004508A1003308A300320895202E
:100B2000031D932D912406305207B200B301B30D7B
:100B30004408A0004508A1003308A30032089D2006
:100B4000031DA32D5124FA305207B200FF300318C1
:100B5000013EB3004408A0004508A1003308A300EB
:100B600032089520031DB52D91244408A0004508A6
:100B7000A10001307E20CC004408A0004508A1005F
:100B800000307E20CD00CF015010080083160511E3
:100B900085118312051585110130A3002C305D20CD
:100BA0000A305C208316051664008312051ADA2DBC
:100BB000C90ADB2DC90164000A304902031CD02D8B
:100BC0000511851164305C200511851564305C20A9
:100BD000C901C601C7010A305C20C60A0319C70A49
:100BE0008316051664008312051AF82DC90AF92D1B
:100BF000C90164000A304902031CEB2DC90105112B
:100C00008511831602309B008312470850208316FB
:100C100003309B0083124608502005158511C00142
:100C2000C1010A305C20C00A0319C10A83160516E7
:100C300003108312470CB300460CB2004008A0001A
:100C40004108A1003308A30032089D20031D112E86
:060C5000051185110800EA
:02400E00653F0C
:00000001FF
